:0B000E00010900010A00C100010814F4
:1001DE00EFFD7C007E017FCD120173C3E49FFFE42F
:1001EE009EAD07FF3395E053917F53927FD2008FE0
:1001FE008D8D8B8F098D0AD28EE4F58CF58AD28C7B
:01020E0022CD
:03001B00020232AC
:10023200C0D0C28E30000DA297B3929785098D85EA
:070242000A8BD28ED0D032EE
:03000B0002020FDF
:04020F00C0E0C0D0BB
:10021300C28C1508E508D39400400A758C00758AD2
:0A02230000D28C8005750814C2009B
:05022D00D0D0D0E0324A
:10001E00D2A9D2AB758911D2AFE4F50BF50CAE0BAC
:10002E00AF0CE4FCFD7BFF7AFFF9F8D31201C84058
:10003E000A050CE50C70E7050B80E37F011201DE6B
:10004E00E4F50BF50CAE0BAF0CE4FCFD7BFF7AFF79
:10005E00F9F8D31201C8400A050CE50C70E7050B40
:10006E0080E37F011201DEE4F50BF50CAE0BAF0C55
:10007E00E4FCFD7BFF7AFFF9F8D31201C8400A05B4
:10008E000CE50C70E7050B80E37F011201DEE4F551
:10009E000BF50CAE0BAF0CE4FCFD7BFF7AFFF9F811
:1000AE00D31201C8400A050CE50C70E7050B80E37E
:1000BE007F011201DEE4F50BF50CAE0BAF0CE4FC88
:1000CE00FD7BFF7AFFF9F8D31201C8400A050CE553
:0900DE000C70E7050B80E380FEC5
:030000000200E714
:0C00E700787FE4F6D8FD75812002012E20
:10017300BC000BBE0029EF8DF084FFADF022E4CC70
:10018300F875F008EF2FFFEE33FEEC33FCEE9DEC39
:10019300984005FCEE9DFE0FD5F0E9E4CEFD22ED7F
:1001A300F8F5F0EE8420D21CFEADF075F008EF2FC9
:1001B300FFED33FD4007985006D5F0F222C398FDBA
:0501C3000FD5F0EA2257
:1001C800EB9FF5F0EA9E42F0E99D42F0EC6480C8AE
:0601D80064809845F0224E
:1000F30002001EE493A3F8E493A34003F68001F205
:1001030008DFF48029E493A3F85407240CC8C3330D
:10011300C4540F4420C8834004F456800146F6DFDC
:10012300E4800B010204081020408090000EE47E5E
:10013300019360BCA3FF543F30E509541FFEE493D1
:10014300A360010ECF54C025E060A840B8E493A398
:10015300FAE493A3F8E493A3C8C582C8CAC583CAC3
:10016300F0A3C8C582C8CAC583CADFE9DEE780BE7B
:0100190000E6
:00000001FF
